:103EDB00C108C187C106C105C102C183C100C101AF
:105A120030B30930B2037F28227F292230B2037FBC
:055A22002A227F2B2267
:105884009004BAE0FEA3E0FF9004C0E0FCA3E0FDB6
:0F589400EF4E700BD3ED94FFEC94004002D20561
:0158A30022E2
:100C9A0075FFDE75FFADE4F5E6F5E71251AEA2A6E3
:100CAA00B392061252FE12308F12534C125A128FFE
:100CBA001FC2A7900575E025E025E02457F582E4D8
:100CCA003404F583A3E0FAA3E0FFEA4480FAA90713
:100CDA00900451E4F0A3EAF0A3E9F0900576E02548
:100CEA00E025E02477F582E43404F583A3E0FAA34F
:100CFA00E0FFEA4480FAA907900454E4F0A3EAF07A
:030D0A00A3E9F06A
:030D0D0075252128
:100D1000C20AC208302208200A05125884D20A20CA
:100D200021030211B2C221124D297F01125959EF3C
:080D3000603B300327E4F526C7
:100D380074FFF527F528E5281528AE277002152732
:080D4800D39400EE940050EE7C
:100D50000526E526B480E1123FFFC20390057BE043
:100D60002402FF1257A37F0112562AD2017F0412D8
:100D700053DAEF601B90058FE004F0C39403400248
:100D8000E4F090058FE0FF9004F4F012574FD20882
:100D90007F051253DAEF601B90058EE004F0C394D8
:100DA000034002E4F090058EE0FF9004F5F0125647
:100DB00096D2087F071253DAEF601B90057BE004A0
:100DC000F0C394084002E4F090057BE0FF9004F348
:100DD000F01257A3D208121A038F25900599E065E7
:100DE00025600DE525F090058CE0FD124F38D20806
:100DF000125A128F1FE4FF125959EF6013E4FF12C9
:100E0000562A2002097D15AF1F1259ACD202D2001A
:100E1000E4FF1253DAEF601FC202300004C2008008
:100E20001690058CE06401F0FD900599E0FF124FEB
:100E300038124B26020D10124DB1EF6002D2087F1E
:100E4000011253DAEF6022300104C201801B9005C9
:100E50008DE004F0C394044002E4F090058DE0FFBF
:100E60009004F2F01258A4D20812591E7D157F0189
:100E7000122E007D0E7F0A122E007D067F08122E94
:100E8000007D037F09122E007D17E4FF122E007DE6
:100E9000167F02122E007D147F03122E00E4FD7FC8
:100EA00004122E007D017F05122E007D057F0612A3
:100EB0002E007D027F07122E007D0D7F0B122E006B
:100EC0009005A2E0640160030211A9301C73900533
:100ED0009CE0B4F7081258C4C21C0211A49005ACDF
:100EE000A3E0FAA3E04A70030211A4301B0B9005A3
:100EF0009DE09005ABF00211A49005ABE0FF9005DA
:100F00009DE0C454F0FEEF4E9005ABF0C39005A9F0
:100F1000E0940840030211A47A0579AC7B019005A6
:100F2000ABE0FD121A1B9005ADE475F00112380F0D
:100F30009005AAE004F070069005A9E004F0021103
:0C0F4000A490059CE064F06003020FEB3D
:100F4C00A3E0FFC4135403FE90053FF0EFA2E6921A
:100F5C000B540F900540F0900599E06E6006200B45
:100F6C00030211A4D21C125AE4900540E0FF25E0C4
:100F7C0025E0245AF582E43404F583E0FEB4201C09
:100F8C00EF25E025E02457F582E43404F583A3E053
:100F9C00FAA3E0FDEA547FFAA9058021EEB4302AC9
:100FAC00900540E025E025E02457F582E43404F573
:100FBC0083A3E0FAA3E0FFEA4480FAA9079005AC0A
:100FCC00E4F0A3EAF0A3E9F080099005ACE4F0A307
:0C0FDC00F0A3F0C21BE49005A9F0A3F004
:100FE8000211A490059CE06431703DA3E0651F7078
:100FF800371256C950FBAF1F125A6090059EE090F9
:1010080004D7F090059FE09004D6F09005A0E090FA
:101018000508F09005A1E0900507F0123605125674
:10102800C950FBAF1F125A5190059CE06432703DC5
:10103800A3E0651F70371256C950FBAF1F125A60E4
:1010480090059EE09004D7F090059FE09004D6F0BC
:101058009005A0E0900508F09005A1E0900507F044
:10106800123C0E1256C950FBAF1F125A5190059CE4
:10107800E0642D703CA3E0651F70361256C950FB22
:10108800AF1F125A6090059EE09004D3F090059F20
:10109800E09004D4F09005A0E09004D5F01256C971
:1010A800400512472B80F61256C950FBAF1F125A43
:1010B8005190059CE0642E703AA3E0651F703412CD
:1010C80056C950FBAF1F125A6090059EE09004D39A
:1010D800F090059FE09004D4F09005A0E09004D52E
:1010E800F01256C950FB1248061256C950FBAF1FE2
:1010F800125A5190059CE0FFB40B02D20490058C63
:10110800E06068EF20E764A2AF9209C2AF90059C47
:10111800E014604804705090059DE0FF125AD29088
:101128000599E0FF90058CE0FD124F3890058DE0A1
:10113800FF1258A490057BE0FF1257A390058FE09B
:10114800FF12574F90057BE0FF1257A390058EE0E2
:10115800FF125696125AC712308F800890059DE0EC
:10116800FF125A99124B26A20992AF90059CE0B43F
:10117800141290058C7401F0900599E0FF7D01121E
:101188004F38D20890059CE0B41511E490058CF016
:10119800900599E0FFE4FD124F38D208E49005A2CB
:1011A800F0300806124B26125A6F200703020D1062
:0511B800124B26C207E6
:0311BD00020D1010
:103EEB0043049C0104B243049F0104C20108000176
:103EFB00090041049900010A00020B000242049AD6
:063F0B000000C119C11AFB
:105A2700AF84E4F58475E881F5BBF5BA75BCA84386
:045A3700E7028F846F
:015A3B002248
:1059E100AF8475840275E888E4F5BAF5BB75BCC06F
:0859F10043BC0143E7108F8461
:0159F900228B
:031A300002434529
:10434500C0E0C083C082C0D075D000C000C005C029
:0343550006C00798
:10435800C2EDE50925E024A2F582E43404F583E002
:10436800FEA3E0FFC3E5BE9F900570F0E5BF9E90F9
:10437800056FF0E0FEA3E0FFD39400EE6480948024
:104388004045AD09E508A805088002C313D8FC30EC
:10439800E0028053D3EF9480EE648094825003024D
:1043A8004438E50925E024A2F582E43404F583E5E0
:1043B800BFF0A3E5BEF0AF097401A807088002C3E7
:1043C80033D8FC4208806990056FE0FEA3E0FFC384
:1043D800EE648094805059AD09E508A8050880026C
:1043E800C313D8FC20E016E50925E024A2F582E4F1
:1043F8003404F583E5BFF0A3E5BEF08033C3EF9442
:1044080080EE6480947D5028E50925E024A2F58299
:10441800E43404F583E5BFF0A3E5BEF0AF09740109
:10442800A807088002C333D8FCFFC3E5089FF50836
:0A4438000509E5095407F509F5BB75
:10444200D007D006D005D000D0D0D082D083D0E023
:014452003237
:031A3900023D7AF1
:103D7A00C0E0C0F0C083C082C0D075D000C000C00F
:0D3D8A0001C002C003C004C005C006C00790
:103D9700C2EDAFBE8F4B8F4C90049CE0FBA3E0FAC3
:103DA700A3E0F975F002E50AA4F58285F0831238DD
:103DB7003BFFAEF0C3E54C9F900572F0E54B9E903C
:103DC7000571F0E0FEA3E0FFD39400EE64809480D9
:103DD7004057AD0A900499E0FCA805088002C31378
:103DE700D8FC30E0028065D3EF9464EE6480948061
:103DF7005003023EB690049CE0FBA3E0FAA3E0F96F
:103E070075F002E50AA4F58285F083E54B854CF051
:103E1700123892900499E0FFAE0A7401A806088050
:103E270002C333D8FC4F023EB2900571E0FEA3E017
:103E3700FFC3EE648094805076AD0A900499E0FC4D
:103E4700A805088002C313D8FC20E02090049CE05A
:103E5700FBA3E0FAA3E0F975F002E50AA4F5828571
:103E6700F083E54B854CF01238928043C3EF949C66
:103E7700EE6480947F503890049CE0FBA3E0FAA3A3
:103E8700E0F975F002E50AA4F58285F083E54B8534
:103E97004CF0123892900499E0FFAE0A7401A8061C
:103EA700088002C333D8FCFEC3EF9E900499F00547
:093EB7000AE50A5407F50AF5BBFF
:103EC000D007D006D005D004D003D002D001D00056
:0B3ED000D0D0D082D083D0F0D0E03200
:031A15000215793E
:10157900C0E0C0F0C083C082C0D075D000C000C038
:0D15890001C002C003C004C005C006C007B9
:10159600C2FFE50C20E0030218A5AF9BEF420EE563
:1015A6000C6403450B7020E50EC4F8540FC868FFA1
:1015B600E50DC454F048F990049FE0FBA3E0FAA3BC
:1015C600E0C98FF0123873E50C640F450B60030217
:1015D60016E6E50C24FFFFE50B34FFC313FEEF13FD
:1015E60024FEFFEE34FFFEEF25E0FFEE33FE90040F
:1015F6009FE0FBA3E0FAA3E0F98F828E8312383BCB
:10160600FFE5F0C4F854F0C868FEEFC4540F48FF75
:10161600C3E50E9FFFE50D9EFE90049AF0A3EFF042
:10162600D39400EE6480948040543019030217ADC1
:10163600D390049BE0940390049AE06480948050D5
:101646000302186AE50EC4F8540FC868FDE50DC418
:1016560054F048FCE50C24FFFFE50B34FFC313FEF2
:10166600EF1324FEFFEE34FFFEEF25E0FFEE338F8F
:1016760082F583EC8DF0123892D21902186AC39063
:10168600049AE064809480400302186A20190302D9
:1016960017ADC390049BE094FD90049AE064809497
:1016A6007F400302186AE50EC4F8540FC868FDE5CA
:1016B6000DC454F048FCE50C24FFFFE50B34FFC3D2
:1016C60013FEEF1324FEFFEE34FFFEEF25E0FFEEE0
:1016D600338F82F583EC8DF0123892C21902186AA4
:1016E600E50C640D450B6003021829E50C24FFFF89
:1016F600E50B34FFC313FEEF1324FEFFEE34FFFEAB
:10170600EF25E0FFEE33FE90049FE0FBA3E0FAA393
:10171600E0F98F828E8312383BFFE5F0C4F854F06F
:10172600C868FEEFC4540F48FFC3E50E9FFFE50DE2
:101736009EFE90049AF0A3EFF0D39400EE6480949A
:10174600804053301A02805FD390049BE09403904C
:10175600049AE064809480500302186AE50EC4F887
:10176600540FC868FDE50DC454F048FCE50C24FF91
:10177600FFE50B34FFC313FEEF1324FEFFEE34FF29
:10178600FEEF25E0FFEE338F82F583EC8DF0123805
:1017960092D21A02186AC390049AE0648094804038
:1017A6000302186A201A32E50EC4F8540FC868FD01
:1017B600E50DC454F048FCE50C24FFFFE50B34FFAF
:1017C600C313FEEF1324FEFFEE34FFFEEF25E0FF0A
:1017D600EE338F82F583021864C390049BE094FD78
:1017E60090049AE06480947F507AE50EC4F8540F12
:1017F600C868FDE50DC454F048FCE50C24FFFFE580
:101806000B34FFC313FEEF1324FEFFEE34FFFEEF8F
:1018160025E0FFEE338F82F583EC8DF0123892C20D
:101826001A8041E50EC4F8540FC868FDE50DC4548E
:10183600F048FCE50C24FFFFE50B34FFC313FEEF75
:101846001324FEFFEE34FFFEEF25E0FFEE33FE909D
:10185600049FE0FBA3E0FAA3E0F98F828E83EC8D70
:10186600F0123892050CE50C7002050BD39413E5C3
:101876000B9400400E750B00750C02750F00751069
:10188600848038E50C24FEFFE50B34FFFEEF78027A
:10189600C333CE33CED8F98E0F4484F510801CAFF7
:1018A6009B750D008F0EE50E750E00F50D750F007C
:0B18B600751000050CE50C7002050B1E
:1018C100D007D006D005D004D003D002D001D0007B
:0B18D100D0D0D082D083D0F0D0E03225
:103F1100C1214105900041059AFF4805910000002B
:053F210000000000009B
:104D2900900541E5B0F0E4A3F0900542E0FFC3949B
:034D3900085074AB
:104D3C007401A807088002C333D8FCF529900541FB
:104D4C00E0552924FF920C90059AE0FB5529603020
:104D5C00900590E0FE552924FF920D200C3E200D6D
:104D6C003BE5294EF0E529F4FFEB5F90059AF090B6
:0E4D7C000542E02491F582E43405F583E4F06D
:104D8A00801C300C0990059AE04529F080109005A6
:0E4D9A0042E02491F582E43405F583E004F054
:084DA800900542E004F0808256
:014DB00022E0
:1053DA007401A807088002C333D8FCFF900541F086
:1053EA00900590E0FE5F6010900541E0FF90059AFD
:1053FA00E05F60047F0180027F00900542EFF06069
:10540A000A900541E0F45E900590F0900542E0FFB5
:01541A00226F
:02562A00AB07CC
:10562C007401A807088002C333D8FC900541F090A0
:10563C000590E0FE900541E0FDF4FCEE5C900590D9
:10564C00F090059AE04DF074912BF582E43405F559
:03565C0083E4F0F4
:01565F002228
:1059590074912FF582E43405F583E0D3940840036C
:0B596900D38001C3920DA20DE433FFB8
:015974002210
:0E1A0300900541E5B0F0E0540C1313543FFF82
:011A110022B2
:0A5AA600AF84E4F58475D4978F8473
:015AB00022D3
:0A5AB100AF8475840175D4978F84CB
:015ABB0022C8
:10502500AB84AAB1A2AF920D8F3E8E3D8D3C8C3BD9
:10503500AE3DAF3E787DA60608A60753B10FE53C09
:10504500700543B110801BE53D30E70543B1308065
:105055001143B120433D80AE3DAF3E787DA60608A5
:10506500A607E4F584C2AF43B701758F03787DE6E3
:10507500FE08E6F5828E83E4F053B7FEF58FA20DA8
:0650850092AF8AB18B849A
:01508B002202
:104FB000AB84AAB1A2AF920D8F4A8E498D488C471F
:104FC000AF46EF3395E0FEEFF44E6050AE49AF4A86
:104FD000787DA60608A60753B10FE548700543B1D2
:104FE00010801BE54930E70543B130801143B12003
:104FF000434980AE49AF4A787DA60608A607E4F586
:1050000084C2AF43B701758F01787DE6FE08E6F5EF
:10501000828E83E546F053B7FEE4F58FA20D92AF82
:045020008AB18B8442
:015024002269
:0E5397008B2D8A2E892F8F338E328D318C30E4
:1053A500E4F536F537C3E5379535E53695345024BC
:1053B50078301238D51252AEAB2D052FE52FAA2E17
:1053C5007002052E14F9EF1237FD0537E53770D554
:0453D500053680D148
:0153D90022B1
:1052AE00AB84AAB18F3B8E3A8D398C38AE3AAF3B78
:1052BE00787DA60608A60753B10FE539700543B1F0
:1052CE0010801BE53A30E70543B130801143B12021
:1052DE00433A80AE3AAF3B787DA60608A607787DA6
:0F52EE00E6FE08E6F5828E83E493FF8AB18B8497
:0152FD00228E
:0B5ABC00AF01AE027C00E4FD025025AB
:021A1B008D41FB
:0E1A1D00AF01AE027C00E4FD854146024FB0F1
:10541B008E3B8F3C8C3D8D3E8A3F8B40E540453F1C
:10542B00602BAA3BA93C7B01853E82853D83E0FD39
:10543B00121A1BE54015407002153F053EE53E7004
:0E544B0002053D053CE53C70D3053B80CF22B9
:065AE400E4F57BF57C22D5
:1058C400AA7BA97C7BFF125ABC7C007D007B007AFA
:0E58D40004AF7CAE7B12541BE4F57BF57C2206
:064E37008E368F378D3826
:104E3D00EE54FCFEE57C7003EE657B605CE57C4525
:104E4D007B60031258C4E53654FCF57B757C00F588
:104E5D0039857C3A7E007F0090056D7403F0A37454
:104E6D00FFF0053AE53AAC397002053914F5828C3C
:104E7D0083E493FD0FEFAA0670010E14F5828A8369
:104E8D00EDF090056EE024FFF090056DE034FFF03D
:104E9D00E0B4FFCEA3E0B4FFC9E5365403FE7400C1
:0C4EAD002537F58274003EF583E538F0EF
:014EB90022D6
:1054D4008E2F8F308B318A328933E5351535AE34D2
:1054E400700215344E60230530E530AE2F7002058E
:1054F4002F14FFAB310533E533AA327002053214A1
:0B550400F91237B7FD124E3780D0229D
:1051AE00752927752A10E52A152AAE2970021529A8
:0851BE00D39400EE940050EEC2
:1051C6007D017F0412514E12593C125A3C1248D8A6
:1051D600125AA6125AB11259E1125A2775F7041239
:1051E60054977FB87E2E1258E27F997E5712584008
:1051F6007FD77E05125862D2AFE4F58475D10322BB
:10514E00AE8475840F758C20E4F58475EF06758436
:10515E000F758A83F59775840F758904F58475B775
:10516E003075840F4389018D8D758F018F8EFDFCF7
:10517E000DBD00010CE4B505F7ECB401F343890253
:10518E00E58920E4120DEDAA0470010C14D39400ED
:0F519E00EA6480948140E9759702E4F58A8E8473
:0151AD0022DF
:10593C00AF8475840F75E10375E34075AD0175A5F2
:0C594C000175A6BF75A04075A4E78F840C
:01595800222C
:105A3C00E4F584759A73759D1A43E60175F801C2F5
:055A4C0087759B842218
:0D48D800AE8475840F20060302496BC29068
:1048E500752B00752C10E52C152CAC2B7002152B97
:0848F500D39400EC940050EE96
:0648FD007F28C286C2857F
:10490300752B00752C10E52C152CAC2B7002152B78
:08491300D39400EC940050EE77
:02491B00D28543
:10491D00752B00752C10E52C152CAC2B7002152B5E
:08492D00D39400EC940050EE5D
:02493500DFC8D9
:10493700752B00752C10E52C152CAC2B7002152B44
:08494700D39400EC940050EE43
:02494F00D29004
:10495100752B00752C10E52C152CAC2B7002152B2A
:0A496100D39400EC9400403C80EC7D
:06496B007F28C286C28510
:10497100752B00752C10E52C152CAC2B7002152B0A
:08498100D39400EC940050EE09
:02498900D285D5
:10498B00752B00752C10E52C152CAC2B7002152BF0
:08499B00D39400EC940050EEEF
:0449A300DFC88E8457
:0149A70022ED
:1058E200AD84E4F584F5C875C908C39FFFE49EF54D
:0D58F200CB8FCA74FFF5CDF5CCD2CA8D84E2
:0158FF002286
:10584000AD84758401E4F5C875C908C39FFFE49E63
:10585000F5CB8FCA74FFF5CDF5CC43E701D2CA8DE5
:0158600084C3
:015861002224
:10586200AD84758402E4F5C875C908C39FFFE49E40
:10587200F5CB8FCA74FFF5CDF5CC43E704D2CA8DC0
:0158820084A1
:015883002202
:101A3C000000000300060009000C000F0012001546
:101A4C000019001C001F002200250028002B002F6D
:101A5C00003200350038003B003E00410045004894
:101A6C00004B004E005100540057005A005E0061BC
:101A7C0000640067006A006D007000730077007AE4
:101A8C00007D0080008300860089008C008F00930D
:101A9C0000960099009C009F00A200A500A800AB36
:101AAC0000AE00B200B500B800BB00BE00C100C45F
:101ABC0000C700CA00CD00D000D300D700DA00DD8B
:101ACC0000E000E300E600E900EC00EF00F200F5B6
:101ADC0000F800FB00FE010101040107010A010DE1
:101AEC00011001140117011A011D01200123012607
:101AFC000129012C012F013201350138013B013E36
:101B0C000141014401470149014C014F015201556A
:101B1C000158015B015E016101640167016A016D9D
:101B2C000170017301760179017C017E01810184D0
:101B3C000187018A018D0190019301960199019B06
:101B4C00019E01A101A401A701AA01AD01AF01B23F
:101B5C0001B501B801BB01BE01C001C301C601C979
:101B6C0001CC01CE01D101D401D701DA01DC01DFB6
:101B7C0001E201E501E801EA01ED01F001F301F5F3
:101B8C0001F801FB01FD0200020302060208020B30
:101B9C00020E0210021302160218021B021E022071
:101BAC00022302260228022B022E023002330236B6
:101BBC000238023B023D0240024302450248024AFF
:101BCC00024D024F025202550257025A025C025F4A
:101BDC000261026402660269026B026E0270027399
:101BEC0002750278027A027D027F028102840286EB
:101BFC000289028B028E0290029202950297029A3F
:101C0C00029C029E02A102A302A502A802AA02AD96
:101C1C0002AF02B102B302B602B802BA02BD02BFF1
:101C2C0002C102C402C602C802CA02CD02CF02D14E
:101C3C0002D302D502D802DA02DC02DE02E002E3B1
:101C4C0002E502E702E902EB02ED02F002F202F415
:101C5C0002F602F802FA02FC02FE0300030203047D
:101C6C0003070309030B030D030F031103130315E0
:101C7C0003170319031B031D031F03210322032452
:101C8C0003260328032A032C032E033003320334C8
:101C9C00033603370339033B033D033F0341034240
:101CAC00034403460348034A034B034D034F0351BC
:101CBC0003530354035603580359035B035D035F3B
:101CCC00036003620364036503670369036A036CBF
:101CDC00036D036F03710372037403750377037849
:101CEC00037A037C037D037F0380038203830385D4
:101CFC00038603880389038B038C038D038F039066
:101D0C00039203930395039603970399039A039BFA
:101D1C00039D039E039F03A103A203A303A503A694
:101D2C0003A703A803AA03AB03AC03AD03AF03B033
:101D3C0003B103B203B303B503B603B703B803B9D6
:101D4C0003BA03BC03BD03BE03BF03C003C103C27C
:101D5C0003C303C403C503C603C703C803C903CA2B
:101D6C0003CB03CC03CD03CE03CF03D003D103D2DB
:101D7C0003D303D403D503D603D703D703D803D98E
:101D8C0003DA03DB03DC03DC03DD03DE03DF03E048
:101D9C0003E003E103E203E303E303E403E503E508
:101DAC0003E603E703E703E803E903E903EA03EBCC
:101DBC0003EB03EC03ED03ED03EE03EE03EF03EF94
:101DCC0003F003F003F103F103F203F203F303F363
:101DDC0003F403F403F503F503F603F603F703F733
:101DEC0003F703F803F803F803F903F903F903FA0B
:101DFC0003FA03FA03FB03FB03FB03FB03FC03FCE7
:101E0C0003FC03FC03FD03FD03FD03FD03FD03FEC7
:101E1C0003FE03FE03FE03FE03FE03FE03FF03FFAC
:101E2C0003FF03FF03FF03FF03FF03FF03FF03FF96
:101E3C0003FF03FF03FF03FF03FF03FF03FF03FF86
:101E4C0003FF03FF03FF03FE03FE03FE03FE03FE7B
:101E5C0003FE03FE03FD03FD03FD03FD03FD03FC75
:101E6C0003FC03FC03FC03FB03FB03FB03FB03FA74
:101E7C0003FA03FA03F903F903F903F803F803F877
:101E8C0003F703F703F703F603F603F503F503F47F
:101E9C0003F403F303F303F203F203F103F103F08E
:101EAC0003F003EF03EF03EE03EE03ED03ED03EC9E
:101EBC0003EB03EB03EA03E903E903E803E703E7B6
:101ECC0003E603E503E503E403E303E303E203E1D1
:101EDC0003E003E003DF03DE03DD03DC03DC03DBF1
:101EEC0003DA03D903D803D703D703D603D503D416
:101EFC0003D303D203D103D003CF03CE03CD03CC42
:101F0C0003CB03CA03C903C803C703C603C503C471
:101F1C0003C303C203C103C003BF03BE03BD03BCA1
:101F2C0003BA03B903B803B703B603B503B303B2DB
:101F3C0003B103B003AF03AD03AC03AB03AA03A817
:101F4C0003A703A603A503A303A203A1039F039E58
:101F5C00039D039B039A039903970396039503939D
:101F6C0003920390038F038D038C038B03890388E7
:101F7C0003860385038303820380037F037D037C35
:101F8C00037A037803770375037403720371036F89
:101F9C00036D036C036A03690367036503640362DF
:101FAC000360035F035D035B03590358035603543B
:101FBC0003530351034F034D034B034A034803469A
:101FCC00034403420341033F033D033B03390337FF
:101FDC000336033403320330032E032C032A032865
:101FEC000326032403220321031F031D031B0319D0
:101FFC000317031503130311030F030D030B03093D
:10200C00030703040302030002FE02FC02FA02F8B7
:10201C0002F602F402F202F002ED02EB02E902E730
:10202C0002E502E302E002DE02DC02DA02D802D5AB
:10203C0002D302D102CF02CD02CA02C802C602C428
:10204C0002C102BF02BD02BA02B802B602B302B1AB
:10205C0002AF02AD02AA02A802A502A302A1029E2F
:10206C00029C029A0297029502920290028E028BB7
:10207C000289028602840281027F027D027A027842
:10208C00027502730270026E026B026902660264D0
:10209C000261025F025C025A025702550252024F61
:1020AC00024D024A0248024502430240023D023BF5
:1020BC000238023602330230022E022B022802268C
:1020CC0002230220021E021B021802160213021027
:1020DC00020E020B020802060203020001FD01FBC4
:1020EC0001F801F501F301F001ED01EA01E801E568
:1020FC0001E201DF01DC01DA01D701D401D101CE0B
:10210C0001CC01C901C601C301C001BE01BB01B8AC
:10211C0001B501B201AF01AD01AA01A701A401A152
:10212C00019E019B0199019601930190018D018AF9
:10213C00018701840181017E017C017901760173A3
:10214C000170016D016A016701640161015E015B4F
:10215C00015801550152014F014C014901470144FD
:10216C000141013E013B013801350132012F012CA7
:10217C000129012601230120011D011A0117011457
:10218C000110010D010A01070104010100FE00FB11
:10219C0000F800F500F200EF00EC00E900E600E3C7
:1021AC0000E000DD00DA00D700D300D000CD00CA7B
:1021BC0000C700C400C100BE00BB00B800B500B22F
:1021CC0000AE00AB00A800A500A2009F009C0099E7
:1021DC0000960093008F008C00890086008300809D
:1021EC00007D007A007700730070006D006A006754
:1021FC0000640061005E005A005700540051004E0C
:10220C00004B004800450041003E003B00380035C3
:10221C000032002F002B002800250022001F001C7C
:10222C00001900150012000F000C00090006000335
:10223C000000FFFCFFF9FFF6FFF3FFF0FFEDFFEAF4
:10224C00FFE6FFE3FFE0FFDDFFDAFFD7FFD4FFD0AF
:10225C00FFCDFFCAFFC7FFC4FFC1FFBEFFBAFFB768
:10226C00FFB4FFB1FFAEFFABFFA8FFA5FFA1FF9E20
:10227C00FF9BFF98FF95FF92FF8FFF8CFF88FF85D8
:10228C00FF82FF7FFF7CFF79FF76FF73FF70FF6C8F
:10229C00FF69FF66FF63FF60FF5DFF5AFF57FF5446
:1022AC00FF51FF4DFF4AFF47FF44FF41FF3EFF3BFD
:1022BC00FF38FF35FF32FF2FFF2CFF28FF25FF22B1
:1022CC00FF1FFF1CFF19FF16FF13FF10FF0DFF0A66
:1022DC00FF07FF04FF01FEFEFEFBFEF8FEF5FEF21B
:1022EC00FEEFFEEBFEE8FEE5FEE2FEDFFEDCFED9D5
:1022FC00FED6FED3FED0FECDFECAFEC7FEC4FEC186
:10230C00FEBEFEBBFEB8FEB6FEB3FEB0FEADFEAA30
:10231C00FEA7FEA4FEA1FE9EFE9BFE98FE95FE92DD
:10232C00FE8FFE8CFE89FE86FE83FE81FE7EFE7B8A
:10233C00FE78FE75FE72FE6FFE6CFE69FE66FE6434
:10234C00FE61FE5EFE5BFE58FE55FE52FE50FE4DDB
:10235C00FE4AFE47FE44FE41FE3FFE3CFE39FE3681
:10236C00FE33FE31FE2EFE2BFE28FE25FE23FE2024
:10237C00FE1DFE1AFE17FE15FE12FE0FFE0CFE0AC7
:10238C00FE07FE04FE02FDFFFDFCFDF9FDF7FDF46A
:10239C00FDF1FDEFFDECFDE9FDE7FDE4FDE1FDDF09
:1023AC00FDDCFDD9FDD7FDD4FDD1FDCFFDCCFDC9A4
:1023BC00FDC7FDC4FDC2FDBFFDBCFDBAFDB7FDB53B
:1023CC00FDB2FDB0FDADFDAAFDA8FDA5FDA3FDA0D0
:1023DC00FD9EFD9BFD99FD96FD94FD91FD8FFD8C61
:1023EC00FD8AFD87FD85FD82FD80FD7EFD7BFD79EF
:1023FC00FD76FD74FD71FD6FFD6DFD6AFD68FD657B
:10240C00FD63FD61FD5EFD5CFD5AFD57FD55FD5202
:10241C00FD50FD4EFD4CFD49FD47FD45FD42FD4087
:10242C00FD3EFD3BFD39FD37FD35FD32FD30FD2E0A
:10243C00FD2CFD2AFD27FD25FD23FD21FD1FFD1C87
:10244C00FD1AFD18FD16FD14FD12FD0FFD0DFD0B03
:10245C00FD09FD07FD05FD03FD01FCFFFCFDFCFB7B
:10246C00FCF8FCF6FCF4FCF2FCF0FCEEFCECFCEAF8
:10247C00FCE8FCE6FCE4FCE2FCE0FCDEFCDDFCDB66
:10248C00FCD9FCD7FCD5FCD3FCD1FCCFFCCDFCCBD0
:10249C00FCC9FCC8FCC6FCC4FCC2FCC0FCBEFCBD38
:1024AC00FCBBFCB9FCB7FCB5FCB4FCB2FCB0FCAE9C
:1024BC00FCACFCABFCA9FCA7FCA6FCA4FCA2FCA0FD
:1024CC00FC9FFC9DFC9BFC9AFC98FC96FC95FC9359
:1024DC00FC92FC90FC8EFC8DFC8BFC8AFC88FC87AF
:1024EC00FC85FC83FC82FC80FC7FFC7DFC7CFC7A04
:1024FC00FC79FC77FC76FC74FC73FC72FC70FC6F52
:10250C00FC6DFC6CFC6AFC69FC68FC66FC65FC649C
:10251C00FC62FC61FC60FC5EFC5DFC5CFC5AFC59E2
:10252C00FC58FC57FC55FC54FC53FC52FC50FC4F23
:10253C00FC4EFC4DFC4CFC4AFC49FC48FC47FC4660
:10254C00FC45FC43FC42FC41FC40FC3FFC3EFC3D9A
:10255C00FC3CFC3BFC3AFC39FC38FC37FC36FC35CB
:10256C00FC34FC33FC32FC31FC30FC2FFC2EFC2DFB
:10257C00FC2CFC2BFC2AFC29FC28FC28FC27FC2628
:10258C00FC25FC24FC23FC23FC22FC21FC20FC1F4E
:10259C00FC1FFC1EFC1DFC1CFC1CFC1BFC1AFC1A6E
:1025AC00FC19FC18FC18FC17FC16FC16FC15FC148A
:1025BC00FC14FC13FC12FC12FC11FC11FC10FC10A2
:1025CC00FC0FFC0FFC0EFC0EFC0DFC0DFC0CFC0CB3
:1025DC00FC0BFC0BFC0AFC0AFC09FC09FC08FC08C3
:1025EC00FC08FC07FC07FC07FC06FC06FC06FC05CB
:1025FC00FC05FC05FC04FC04FC04FC04FC03FC03CF
:10260C00FC03FC03FC02FC02FC02FC02FC02FC01CD
:10261C00FC01FC01FC01FC01FC01FC01FC00FC00C8
:10262C00FC00FC00FC00FC00FC00FC00FC00FC00BE
:10263C00FC00FC00FC00FC00FC00FC00FC00FC00AE
:10264C00FC00FC00FC00FC01FC01FC01FC01FC0199
:10265C00FC01FC01FC02FC02FC02FC02FC02FC037F
:10266C00FC03FC03FC03FC04FC04FC04FC04FC0560
:10267C00FC05FC05FC06FC06FC06FC07FC07FC073D
:10268C00FC08FC08FC08FC09FC09FC0AFC0AFC0B15
:10269C00FC0BFC0CFC0CFC0DFC0DFC0EFC0EFC0FE6
:1026AC00FC0FFC10FC10FC11FC11FC12FC12FC13B6
:1026BC00FC14FC14FC15FC16FC16FC17FC18FC187E
:1026CC00FC19FC1AFC1AFC1BFC1CFC1CFC1DFC1E43
:1026DC00FC1FFC1FFC20FC21FC22FC23FC23FC2403
:1026EC00FC25FC26FC27FC28FC28FC29FC2AFC2BBE
:1026FC00FC2CFC2DFC2EFC2FFC30FC31FC32FC3372
:10270C00FC34FC35FC36FC37FC38FC39FC3AFC3B21
:10271C00FC3CFC3DFC3EFC3FFC40FC41FC42FC43D1
:10272C00FC45FC46FC47FC48FC49FC4AFC4CFC4D77
:10273C00FC4EFC4FFC50FC52FC53FC54FC55FC571B
:10274C00FC58FC59FC5AFC5CFC5DFC5EFC60FC61BA
:10275C00FC62FC64FC65FC66FC68FC69FC6AFC6C55
:10276C00FC6DFC6FFC70FC72FC73FC74FC76FC77EB
:10277C00FC79FC7AFC7CFC7DFC7FFC80FC82FC837D
:10278C00FC85FC87FC88FC8AFC8BFC8DFC8EFC9009
:10279C00FC92FC93FC95FC96FC98FC9AFC9BFC9D93
:1027AC00FC9FFCA0FCA2FCA4FCA6FCA7FCA9FCAB17
:1027BC00FCACFCAEFCB0FCB2FCB4FCB5FCB7FCB998
:1027CC00FCBBFCBDFCBEFCC0FCC2FCC4FCC6FCC813
:1027DC00FCC9FCCBFCCDFCCFFCD1FCD3FCD5FCD78D
:1027EC00FCD9FCDBFCDDFCDEFCE0FCE2FCE4FCE602
:1027FC00FCE8FCEAFCECFCEEFCF0FCF2FCF4FCF675
:10280C00FCF8FCFBFCFDFCFFFD01FD03FD05FD07D9
:10281C00FD09FD0BFD0DFD0FFD12FD14FD16FD1840
:10282C00FD1AFD1CFD1FFD21FD23FD25FD27FD2AA5
:10283C00FD2CFD2EFD30FD32FD35FD37FD39FD3B08
:10284C00FD3EFD40FD42FD45FD47FD49FD4CFD4E65
:10285C00FD50FD52FD55FD57FD5AFD5CFD5EFD61C1
:10286C00FD63FD65FD68FD6AFD6DFD6FFD71FD7419
:10287C00FD76FD79FD7BFD7EFD80FD82FD85FD876E
:10288C00FD8AFD8CFD8FFD91FD94FD96FD99FD9BC0
:10289C00FD9EFDA0FDA3FDA5FDA8FDAAFDADFDB00F
:1028AC00FDB2FDB5FDB7FDBAFDBCFDBFFDC2FDC45B
:1028BC00FDC7FDC9FDCCFDCFFDD1FDD4FDD7FDD9A4
:1028CC00FDDCFDDFFDE1FDE4FDE7FDE9FDECFDEFE9
:1028DC00FDF1FDF4FDF7FDF9FDFCFDFFFE02FE042C
:1028EC00FE07FE0AFE0CFE0FFE12FE15FE17FE1A68
:1028FC00FE1DFE20FE23FE25FE28FE2BFE2EFE31A5
:10290C00FE33FE36FE39FE3CFE3FFE41FE44FE47E2
:10291C00FE4AFE4DFE50FE52FE55FE58FE5BFE5E1C
:10292C00FE61FE64FE66FE69FE6CFE6FFE72FE7555
:10293C00FE78FE7BFE7EFE81FE83FE86FE89FE8C8B
:10294C00FE8FFE92FE95FE98FE9BFE9EFEA1FEA4BF
:10295C00FEA7FEAAFEADFEB0FEB3FEB6FEB8FEBBF1
:10296C00FEBEFEC1FEC4FEC7FECAFECDFED0FED327
:10297C00FED6FED9FEDCFEDFFEE2FEE5FEE8FEEB57
:10298C00FEEFFEF2FEF5FEF8FEFBFEFEFF01FF047D
:10299C00FF07FF0AFF0DFF10FF13FF16FF19FF1CA7
:1029AC00FF1FFF22FF25FF28FF2CFF2FFF32FF35D3
:1029BC00FF38FF3BFF3EFF41FF44FF47FF4AFF4DFF
:1029CC00FF51FF54FF57FF5AFF5DFF60FF63FF6627
:1029DC00FF69FF6CFF70FF73FF76FF79FF7CFF7F51
:1029EC00FF82FF85FF88FF8CFF8FFF92FF95FF987A
:1029FC00FF9BFF9EFFA1FFA5FFA8FFABFFAEFFB1A2
:102A0C00FFB4FFB7FFBAFFBEFFC1FFC4FFC7FFCAC9
:102A1C00FFCDFFD0FFD4FFD7FFDAFFDDFFE0FFE3F0
:102A2C00FFE6FFEAFFEDFFF0FFF3FFF6FFF9FFFC17
:102A3C000000010202030404050607070809090A3D
:102A4C000B0C0C0D0E0E0F10111112131414151675
:102A5C00171718191A1A1B1C1D1E1E1F20212122A4
:102A6C002324252526272829292A2B2C2D2D2E2FCA
:102A7C003031323233343536373738393A3B3C3DE6
:102A8C003D3E3F40414243434445464748494A4BFB
:102A9C004B4C4D4E4F505152535455565657585906
:102AAC005A5B5C5D5E5F6061626364656667686902
:102ABC006A6B6C6C6D6E6F707172737475777879FC
:102ACC007A7B7C7D7E7F80818283848586878889E2
:102ADC008A8B8C8E8F9091929394959697989A9BC3
:102AEC009C9D9E9FA0A1A3A4A5A6A7A8A9ABACAD95
:102AFC00AEAFB0B2B3B4B5B6B7B9BABBBCBDBFC05C
:102B0C00C1C2C4C5C6C7C8CACBCCCDCFD0D1D2D414
:102B1C00D5D6D8D9DADBDDDEDFE1E2E3E5E6E7E8BE
:102B2C00EAEBECEEEFF0F2F3F5F6F7F9FAFBFDFE5B
:103F260060200457000000100080002000D0002010
:103F360000E0002000B0002000C0001000D00020EB
:103F460000E00030602004770000001000C0003060
:103F56000080003000E0003000D0003000C00010CB
:103F660000D0002000E00030C115011100C113C1CE
:103F7600144104500002120000021400000116044D
:023F8600C192E6
:031A1200021A367F
:031A3600C2CF32EA
:031A2D000259005B
:09590000C0E0C0D075D000C00762
:0E590900C2CFAF111511EF7005D2217511B686
:07591700D007D0D0D0E03230
:031A33000211C0DD
:1011C000C0E0C0F0C083C082C0D075D000C000C0F5
:0D11D00001C002C003C004C005C006C00776
:1011DD0085B14DC2CF75840312326A90058DE0142E
:1011ED00606224FE700302129C0460030212A9D2F5
:1011FD0012E51254E0FE7F0070047D0180027D0037
:10120D00A20FE4335DFDE4B50708EEB4E0047F0101
:10121D0080027F00EF4D6019E51430E703D38001A4
:10122D00C3920EA218B00E5008751200751300C2AD
:10123D000FA20E9218D3E5139400E51294E0405CD2
:10124D00D20F8058E51220E7047F0180027F00A2B3
:10125D000FE4335FFFE51230E7047E0180027E006C
:10126D00EE4F6018E51430E703D38001C3920EA250
:10127D0018B00E5007A212B39212C20FA20E9218FE
:10128D00D3E5139400E51294E04011D20F800DD2F6
:10129D0012301708751200751300C21790058EE0F5
:1012AD00FD7008D51623751604800330120EE568FF
:1012BD002513F513E5673512F512800DC3E513956A
:1012CD0068F513E5129567F51290058FE0146041EE
:1012DD001460302402704DE51220E711E51325E06E
:1012ED00FFE51233FEEF2401F54FEE801EE51325C9
:1012FD00E0FFE51233FEC374FF9FF54F747F9EF53B
:10130D004E8021E5132401F54FE5123480F54E8012
:10131D0013E51220E708754E7F754FFF8006754E59
:10132D0080754F01854E77854F78300655E57730BE
:10133D00E704D2138002C213A213301401B3503E3E
:10134D009005A4E054FCF0ED700530131980299040
:10135D00058EE0B4022690043AE0FCA3E0FDD394A0
:10136D0000EC948140099005A4E04401F0800DC388
:10137D00EC947F50079005A4E04402F0D207A2132D
:10138D009214758400634E80854ED3854FD275843B
:10139D0003E56C2515F515E56B3514F514E515AE5E
:1013AD00147805CEC313CE13D8F9F54F8E4E25E024
:1013BD00FFE54E33FE743C2FF582741A3EF583E43F
:1013CD0093F54E740193F54F75C303854EC2854F4A
:1013DD00C1856192856291C281C28185964E859546
:1013ED004FE4254FF54F7404354EF54E900575E0DD
:1013FD00FD7014E54FC4F8540FC868F551E54EC49F
:10140D0054F048F5508072EDC39405502453B10F3C
:10141D00900497E042B1900451A3E0FAA3E0F58265
:10142D00E54F25E0FFE54E33FEE5822FF582EA809C
:10143D003953B10F900497E042B19004C4E0FEA37C
:10144D00E07802CEC313CE13D8F9FF90043FE02FFE
:10145D00FF90043EE03E8F82F583E54F25E0FFE5EA
:10146D004E33FEE5822FF582E5833EF583E493F559
:10147D0050740193F551854DB1900576E0FD7014D2
:10148D00E54FC4F8540FC868F553E54EC454F04801
:10149D00F5528072EDC39405502453B10F9004980A
:1014AD00E042B1900454A3E0FAA3E0F582E54F25A4
:1014BD00E0FFE54E33FEE5822FF582EA803953B128
:1014CD000F900498E042B19004C2E0FEA3E07802D0
:1014DD00CEC313CE13D8F9FF90043DE02FFF900437
:1014ED003CE03E8F82F583E54F25E0FFE54E33FE70
:1014FD00E5822FF582E5833EF583E493F552740181
:10150D0093F553854DB1E57930E706757900757A18
:10151D0000C374FF957AF54F747F9579F54E75C3B9
:10152D000E8579C2857AC1855092855191854EC2BD
:10153D00854FC1855292855391C281C281C28185E9
:10154D00CF4E85CE4F634E80758401854ED3854F2A
:01155D00D2BB
:10155E00D007D006D005D004D003D002D001D000E1
:0B156E00D0D0D082D083D0F0D0E0328B
:023F8800C12254
:10308F00E490044EF0A3F09004D8E0FEA3E0FBAA76
:10309F00069004D0E0FEA3E0FFC3EF9BFFEE9AFE85
:1030AF00E49400FDE49400FC9004001238F59004C1
:1030BF00DAE0FEA3E0FBAA069004CCE0FEA3E0FF5B
:1030CF00C3EF9BFFEE9AFEE49400FDE49400FC90A6
:1030DF0004041238F59004DCE0FEA3E0FBAA06908E
:1030EF0004CEE0FEA3E0FFC3EF9BFFEE9AFEE49455
:1030FF0000FDE49400FC9004081238F59004DEE023
:10310F00FEA3E0FBAA069004CAE0FEA3E0FFC3EF14
:10311F009BFFEE9AFEE49400FDE49400FC90040CF7
:10312F001238F59004E0E0FEA3E0FBAA069004A29B
:10313F00E0FEA3E0FFC3EF9BFFEE9AFEE49400FDD9
:10314F00E49400FC9004101238F59004E2E0FEA322
:10315F00E0FBAA069004A4E0FEA3E0FFC3EF9BFFF1
:10316F00EE9AFEE49400FDE49400FC9004141238EF
:10317F00F59004E4E0FEA3E0FBAA069004ACE0FEA9
:10318F00A3E0FFC3EF9BFFEE9AFEE49400FDE494EF
:10319F0000FC9004181238F59004E6E0FEA3E0FB63
:1031AF00AA069004A6E0FEA3E0FFC3EF9BFFEE9AF2
:1031BF00FEE49400FDE49400FC90041C1238F5909A
:1031CF0004E8E0FEA3E0FBAA069004AEE0FEA3E055
:1031DF00FFC3EF9BFFEE9AFEE49400FDE49400FC26
:1031EF009004201238F59004EAE0FEA3E0FBAA0653
:1031FF009004A8E0FEA3E0FFC3EF9BFFEE9AFEE46E
:10320F009400FDE49400FC9004241238F59004EC33
:10321F00E0FEA3E0FBAA069004BEE0FEA3E0FFC31E
:10322F00EF9BFFEE9AFEE49400FDE49400FC900403
:10323F00281238F59004EEE0FEA3E0FBAA069004F6
:10324F00BCE0FEA3E0FFC3EF9BFFEE9AFEE4940009
:0B325F00FDE49400FC90042C0238F504
:10550F009004DAEEF0FDA3EFF0900436CDF0A3EDAA
:10551F00F0AB07AA069004CCE0FEA3E0FFC3EF9B1D
:10552F00FFEE9AFEE49400FDE49400FC9004041254
:0A553F0038F590044FE054FDF0220F
:105582009004ECEEF0A3EFF0900448EEF0A3EFF0FD
:10559200FBAA069004BEE0FEA3E0FFC3EF9BFFEE72
:1055A2009AFEE49400FDE49400FC9004281238F57D
:0855B20090044EE054FBF022CE
:1055BA009004E8EEF0A3EFF0900444EEF0A3EFF0CD
:1055CA00FBAA069004AEE0FEA3E0FFC3EF9BFFEE4A
:1055DA009AFEE49400FDE49400FC9004201238F54D
:0855EA0090044EE054FEF02293
:1055F2009004EAEEF0A3EFF0900446EEF0A3EFF091
:10560200FBAA069004A8E0FEA3E0FFC3EF9BFFEE17
:105612009AFEE49400FDE49400FC9004241238F510
:0856220090044EE054FDF0225B
:042E00008F298D2A5F
:102E0400C20C74017E00A807088005C333CE33CEFC
:102E1400D8F9900542F0EE900541F020222EE52AE3
:102E240025E024A2F582E43404F583E0FEA3E0FF68
:102E3400E52925E02434F582E43404F583EEF0A397
:102E4400EFF074FF90044EF0A3022F10900541E0C0
:102E5400FEA3E0FF90044EE05EFEA3E05F4E70032D
:102E6400022F14E52925E024D8F582E43404F583FF
:102E7400E0FEA3E0FBAA06E52A25E024A2F582E40D
:102E84003404F583E0FEA3E0FFC3EF9BFFEE9AFE5C
:102E9400E49400FDE49400FC74FF7BC0FAF9F8D3D9
:102EA4001238BF5041E52925E024D8F582E43404E2
:102EB400F583E0FEA3E0FBAA06E52A25E024A2F5BB
:102EC40082E43404F583E0FEA3E0FFC3EF9BFFEE4E
:102ED4009AFEE49400FDE49400FCE47B40FAF9F8E3
:102EE400C31238BF5003125A6FE52A25E024A2F515
:102EF40082E43404F583E0FEA3E0FFE52925E02421
:102F040034F582E43404F583EEF0A3EFF07F00227D
:102F1400E52925E024D8F582E43404F583E0FEA312
:102F2400E0FBAA06E52A25E024A2F582E43404F5B0
:102F340083E0FEA3E0FFC3EF9BFFEE9AFEE4940060
:102F4400FDE49400FC9005431238F5E52925E025BD
:102F5400E02400F582E43404F583E0FCA3E0FDA35F
:102F6400E0FEA3E0FF9005471238F5E529B401120D
:102F740090058CE0600CE566643245656004C20C23
:102F8400804A900547E0FCEC33401DE4FFFEFDFC65
:102F9400900543E0F8A3E0F9A3E0FAA3E0FBD31221
:102FA40038BF5004D20C8024E4FFFEFDFC9005479A
:102FB400E0F8A3E0F9A3E0FAA3E0FBD31238BF5092
:102FC4000B900543E0FCEC334002D20C200C0302CE
:102FD4003065900541E0FEA3E0FF90044EE04EF022
:102FE400A3E04FF0E52A25E024A2F582E43404F5B9
:102FF40083E0FEA3E0FFE52925E024D8F582E4344C
:1030040004F583EEF0A3EFF0E52A25E024A2F5828F
:10301400E43404F583E0FEA3E0FFE52925E024344D
:10302400F582E43404F583EEF0A3EFF0E47F40FE90
:10303400FDFC900547E0F8A3E0F9A3E0FAA3E0FB68
:10304400D31238BF501674FF7FC0FEFDFC900547B5
:10305400E0F8A3A3A3E0C31238BF5029125A6F802B
:1030640024E52925E024D8F582E43404F583E0FE40
:10307400A3E0FFE52925E02434F582E43404F58354
:0A308400EEF0A3EFF0A20CE433FF1E
:01308E00221F
:045B01000604020094
:0E3F8A004505A40000000000C1234105A3006E
:10545900E4F52C530707EF5403905B0193FEEFC368
:10546900940450159005A8E0FFEDA806088002C332
:1054790033D8FC4F9005A8F0229005A7E0FFEDA8CE
:0D54890006088002C333D8FC4F9005A7F041
:0154960022F3
:1059C7009005A4E0FE5306F3EF60047F0880027F92
:0959D70004EF42069005A4EEF075
:0159E00022A4
:1049A800900575E0D3940440047F0180027F008F56
:1049B8002B900576E0D3940440047F0180027F00A9
:1049C800AC07E49005A7F0A3F0900575E09004F813
:1049D800F025E025E02457F582E43404F583A3E0CC
:1049E800FAA3E0FFEA4480FAA907900451E4F0A38F
:1049F800EAF0A3E9F0900575E0FF25E025E0245AE8
:104A0800F582E43404F583E0900497F07D011254B4
:104A180059900576E0FF9004F7F00D12545990056F
:104A280076E0FF25E025E02477F582E43404F58379
:104A3800A3E0FAA3E0FBEA4480FAA903900454E453
:104A4800F0A3EAF0A3E9F0EF25E025E0247AF58267
:104A5800E43404F583E0900498F0300607AF04AD21
:044A68002B12599123
:014A6C002227
:0B5AC70090058BE0FF1259C70249A8B0
:104DB100C20CE4F529F52A7F06125959EF60267FC6
:104DC1000612562A20231A90058BE070047F018079
:104DD100027F0090058BEFF09004F6F01259C7D2D4
:104DE1000CD22380267F061253DAEF601E30230493
:104DF100C223801790058BE07005900575800390A4
:104E01000576E004F0E05407F0D20C1249A8300610
:104E11001F900576E0C394054003752A019005753E
:104E2100E0C394054003752901AD29AF2A125991B8
:054E3100A20CE433FFB8
:014E36002259
:104F3800AC079005A6E05430F0ED603730060280EB
:104F480011EC14601214601714601A24037058903E
:104F580005A6E04402F0229005A6E04408F022905D
:104F680005A6E0800A9005A6E04402F04408F04453
:104F780080F022200631EC14601214601714601AB5
:104F8800240370239005A6E04401F0229005A6E0D2
:104F98004404F0229005A6E0800A9005A6E04401AA
:084FA800F04404F04440F02243
:10599100AE079005A6E054CFF0EE6004E04410F0AD
:0B59A100ED60079005A6E04420F02216
:10574F009005A4E0548FF0EF14600F14601424023E
:10575F0070179005A4E04440F0229005A4E0442087
:0A576F00F0229005A4E04410F0229F
:1057A300AD079005A5E054E3F0ED30E004E04410CC
:1057B300F0ED30E1079005A5E04408F0ED30E20795
:0857C3009005A5E04404F0226A
:10569600AD079005A5E054FCF09005A4E0547FF01A
:1056A600ED14600F146014240270179005A4E044F2
:1056B60080F0229005A5E04401F0229005A5E04483
:0356C60002F022CD
:1057CB00AD079005A5E0541FF0ED30E004E04480F8
:1057DB00F0ED30E1079005A5E04440F0ED30E20735
:0857EB009005A5E04420F02226
:1058A400EF14601214601314600824037011E4FFF1
:1058B400800A7F0480067F0180027F021257CB2278
:10591E00857929857A2AAF29C374FF9FC313FF9017
:0D592E0005A3E06F6007EFF053A0C042A09A
:01593B002249
:10581B00EF540314600F146014240270179005A446
:10582B00E054FCF0229005A4E04402F0229005A481
:05583B00E04401F02231
:0A4B2600A98475840F30061AC290AE
:104B3000752900752A10E52A152AAE297002152953
:084B4000D39400EE940050EE46
:024B4800E4FD8A
:0F4B4A0074A42DF582E43405F583E0F529E4FB2E
:104B590074017E00A803088005C333CE33CED8F98B
:104B6900FFE529F582EF558224FF920CA20C92866B
:024B7900C285F3
:104B7B00752A00752B10E52B152BAE2A7002152A02
:084B8B00D39400EE940050EEFB
:024B9300D285C9
:104B9500752A00752B10E52B152BAE2A7002152AE8
:084BA500D39400EE940050EEE1
:044BAD000BBB08A88E
:094BB1000DED6405709330061A45
:104BBA00752900752A10E52A152AAE2970021529C9
:084BCA00D39400EE940050EEBC
:044BD200D290898470
:014BD60022BC
:10534C00300608D290E4FDFF125991900599E0FFC8
:10535C0090058CE0FD124F3890058DE0FF1258A49B
:10536C0090057BE0FF1257A390058FE0FF12574F7B
:10537C00E4FF12581B90057BE0FF1257A390058E9B
:0B538C00E0FF125696125AC7024B2693
:043F98004105A2003D
:0D5A8C001256C950FB7F02124BD7025ADDA3
:0656F700125AF0EF6023DF
:1056FD0075540575559B1256600555E555AC54709E
:10570D0002055414F5828C83EFF0125AF6EF70E611
:03571D007F0122E7
:035720007F0022E5
:1059AC008F298D2A1256C950FB7F0A124BD7AF296B
:0B59BC00124BD7AF2A124BD7025ADD66
:0F5A51008F297F2F124BD7AF29124BD7025ADD67
:0F5A60008F297F30124BD7AF29124BD7025ADD57
:1059FA00000002AB055508000AAB0D55100012ABAA
:085A0A00155518001AAB1D55DB
:023F9C00C11C46
:02411800A907F5
:10411A00E975F00C84ABF07A00E975F00C8424FFA1
:10412A00F55EE434FFF55DEA60030241CAEBB40CC4
:10413A000040030241CA904147F828287302416BA4
:10414A0002417102417702417D02418302418902A3
:10415A00418F02419502419B0241A10241AE0241B7
:10416A00BC7A007B03805D7A007B0480577A007BEF
:10417A000580517A007B06804B7A007B0780457A5E
:10418A00007B08803F7A007B0980397A007B0A80AD
:10419A00337A007B0B802DE4FAFB055EE55E702422
:1041AA00055D80207A007B01055EE55E7016055D7F
:1041BA0080127A007B02055EE55E7008055D800468
:1041CA00E4FEFF22E55EC43354E0FEE4F55C8E5B58
:1041DA00F55AF559EB25E0FFEA33FE74FA2FF5821A
:1041EA0074593EF583E493FE740193FFE4FCFDE504
:1041FA005C2FF55CE55B3EF55BED355AF55AEC351F
:10420A0059F559E9D394674009E4755CFF755BFF7A
:10421A00800BE9C394095009E4F55CF55BF55AF59E
:05422A0059AE5BAF5C22
:01422F00226C
:104453008D1CEF14604A24ECB40B00400302455B4F
:1044630090447175F003A4C58325F0C5837302449A
:104473009202455B0244B50244C60244C90244E6C3
:1044830002450302450E024521024534024547E534
:104493001C75F00A84FF90058DF01258A47F012249
:0F44A300E51C25E0F51CF51DAF1EAE1D12558260
:1044B2007F0122E51C75F00A84FF90057BF01257FC
:1044C200A37F01227F0022E51C75F00A8490058EED
:1044D200F0D3940240037402F090058EE0FF12566E
:1044E200967F0122E51C75F00A8490058FF0D39423
:1044F2000240037402F090058FE0FF12574F7F01D4
:1045020022E51C75F00A849005768009E51C75F099
:104512000A84900575F05407F01249A87F0122E53C
:104522001C25E0F51C751C00AF1C7E001255BA7FDD
:104532000122E51C25E0F51C751C00AF1C7E001253
:1045420055F27F0122E51CFD7C0075F004A4AEF05B
:0F4552002DF566EC3EF56580037F00227F002289
:064561008B548A558956B7
:104567009000011237D0900573F0E0FD540FA3F0CF
:10457700FC900599E0FF74017E00A807088005C339
:1045870033CE33CED8F9FFECFBEF5B24FF9211ED6E
:1045970054F02450603324D0606024F07003024646
:0E45A700482460600302464820110302464883
:1045B500AB54AA55A9569000021237D0FF124118E4
:0945C5008E578F5812550FD217C2
:1045CE008078301175AB54AA55A956900002123757
:1045DE00D0641F70659000031237D0756500F566C4
:1045EE00D39433E56594004051E5661566704B151E
:1045FE00658047301144AB54AA55A956900003125A
:10460E0037D075180025E0F5179000021237D075D7
:10461E00F004A4AEF04218EE4217E5182401F51A84
:10462E00E5173480F519E51AAE197803CEA2E71313
:0C463E00CE13D8F8F51A8E1980007F000A
:01464A00224D
:011A2B00FFBB
:063F9E00C11D4104D20028
:10508C009004F2E090058DF09004F3E090057BF035
:10509C009004F4E090058FF09004F5E090058EF00C
:1050AC009004F6E090058BF09004F7E0900576F014
:1050BC009004F8E0900575F0E4FFEF25E024D8F5B6
:1050CC0082E43404F583E0FCA3E0FDEF25E0243416
:1050DC00F582E43404F583ECF0A3EDF00FBF0DDAA8
:0150EC0022A1
:1050ED0090058DE09004F2F090057BE09004F3F0D4
:1050FD0090058FE09004F4F090058EE09004F5F0AB
:10510D0090058BE09004F6F0900576E09004F7F0B2
:10511D00900575E09004F8F0E4FFEF25E02434F5F8
:10512D0082E43404F583E0FCA3E0FDEF25E024D810
:10513D00F582E43404F583ECF0A3EDF00FBF0DDA46
:01514D00223F
:10525C0090058DE09004F2F090057BE09004F3F063
:10526C0090058FE09004F4F090058EE09004F5F03A
:10527C0090058BE09004F6F0900576E09004F7F042
:10528C00900575E09004F8F0E4FFEF25E024D8F5E4
:10529C0082E43404F583747FF0A374FFF00FBF0D28
:0152AC00E918
:0152AD0022DE
:103FFF00A2AF920CC2AF9004C8E0FCA3E0FDECC4EA
:10400F00F854F0C868FAEDC4540F48FBECC313FE24
:10401F00ED132BFDEE3AFC9004C8E01313543F7ED2
:10402F00002DFFEE3C9004F9F0A3EFF09004C6E0F2
:10403F00FCA3E0FDECC4F854F0C868FAEDC4540FCB
:10404F0048FBECC313FEED132BFDEE3AFC9004C6B8
:10405F00E01313543F7E002DFFEE3C9004FBF0A3C2
:10406F00EFF09004ACE0FFA3E0900501CFF0A3EFD9
:10407F00F09004B8E0FEA3E07802CEC313CE13D8BD
:10408F00F9FF900505EEF0A3EFF09004B4E0FEA366
:10409F00E07802CEC313CE13D8F9FF900503EEF0EC
:1040AF00A3EFF09004C4E0FEA3E0FFC3E49FFF740E
:1040BF00809EFEEF7803CEA2E713CE13D8F8FF90C1
:1040CF0004FDEEF0A3EFF09004C2E0FEA3E0FFC307
:1040DF00E49FFF74809EFEEF7803CEA2E713CE130A
:1040EF00D8F8FF9004FFEEF0A3EFF0125AE47EB879
:1040FF007F007B017A0479F975340075350E1254FF
:08410F00D41258C4A20C92AFB7
:014117002285
:104EBA00E4F52E12525CE49004F9F0A3F0A3F0A3F7
:104ECA00F0900501F0A3F0900505F0A3F09005031A
:104EDA00F0A3F09004FD7480F0A3E4F0A37480F0D2
:104EEA00A3E4F0125AE47EB87F007B017A0479F9D0
:104EFA0075340075350E1254D41258C4125AE4E4AB
:104F0A00F52D75F021E52DA42400F582E5F034A8ED
:104F1A00AF82FE7B017A0479D87534007535211287
:0E4F2A0054D4052DE52DC3941E40D70258C463
:0F5A6F00201D0990058CE06003125A8CD21D2275
:1052FE00901A2BE4936010124EBA7A1A792B7B0116
:07530E00E4FD121A1B8031BF
:105315007AB87900892C8A2B752AFF752900E52C26
:10532500F52CE52BF52BE4F52AF5297B017A047993
:10533500F9AF2CAE2BAD2AAC29F53475350E1253C9
:0153450097D0
:06534600E49004D2F02205
:105779009004D2E075F021A42400F582E5F034A864
:10578900F583AF82FE7C00E4FD7B017A0479D8F5CC
:0957990034753521125397C21D2D
:0157A20022E4
:1057F300125AE49004D2E075F021A42400F582E566
:10580300F034A8AF82FE7B017A0479D87534007531
:0858130035211254D40258C4DF
:065AEA001257F3C21D2259
:0D5A9900AE071250ED9004D2EEF0025AEA72
:0B5AD2009004D2EFF012577902508CC4
:10360500900508E0FB9004D7E0FED39B50030236FB
:10361500E3EE24FFFEE434FF900542F0A3CEF0EB89
:1036250014900541F09004D6E024FFFFE434FFFE3A
:10363500900542E0FCA3E0FDD39FEE6480F8EC64C6
:10364500809840030237B690A80075F021ED123935
:1036550001EC75F021A42583AF82900549F0A3EF15
:10366500F0900541E075F021A42400F974A835F027
:10367500FA90054674FFF0A3EAF0A3E9F0E490059B
:1036850044F0A3F0900546A3E475F001123825FE39
:10369500AFF0900549E475F00112382585F082F503
:1036A50083E493FD124E37900545E004F0700690D3
:1036B5000544E004F0C3900545E09421900544E0FD
:1036C500940040C01258C4900543E004F070069081
:1036D5000542E004F0900541E004F002362A90042A
:1036E500D6E024FFFEE434FF900542F0A3CEF0902F
:1036F5000507E014900541F09004D7E024FFFFE4AE
:1037050034FFFE900542E0FCA3E0FDC39FEE64801C
:10371500F8EC64809850030237B690A80075F02144
:10372500ED123901EC75F021A42583AF829005498E
:10373500F0A3EFF0900541E075F021A42400F974A1
:10374500A835F0FA90054674FFF0A3EAF0A3E9F076
:10375500E4900544F0A3F0900546A3E475F001124A
:103765003825FEAFF0900549E475F001123825853E
:10377500F082F583E493FD124E37900545E004F0A1
:103785007006900544E004F0C3900545E09421904F
:103795000544E0940040C01258C4900543E024FF5E
:1037A500F0900542E034FFF0900541E014F0023658
:0137B500FD16
:0137B60022F0
:103C0E009004D7E014900569F0900508E014900533
:103C1E006AF09004D6E014FF900569E0D39F40034C
:103C2E00023D79A3E075F021A42400F582E5F0347D
:103C3E00A8AF82900546F0A3EFF0E490056BF0A3D9
:103C4E00F090056BE0FEA3E0FFC39421EE940050CC
:103C5E002E900546E475F00112382585F082F58325
:103C6E00E493FD74482FF582E43405F583EDF0906E
:103C7E00056CE004F070CA90056BE004F080C29011
:103C8E00056AE075F021A42400F974A835F0FA90C5
:103C9E00054174FFF0A3EAF0A3E9F0900569E07521
:103CAE00F021A42400F582E5F034A8AF82900544FB
:103CBE00F0A3EFF0E490056BF0A3F0900541A3E4C0
:103CCE0075F001123825FEAFF0900544E475F00151
:103CDE0012382585F082F583E493FD124E37900558
:103CEE006CE004F0700690056BE004F0C390056C78
:103CFE00E0942190056BE0940040C0900569E0755A
:103D0E00F021A42400F974A835F0FA90054174FF4F
:103D1E00F0A3EAF0A3E9F0E490056BF0A3F09005B0
:103D2E006BE0FCA3E0FDC39421EC9400502D9005B4
:103D3E0041A3E475F001123825FEAFF074482DF55D
:103D4E0082E43405F583E0FD124E3790056CE004F5
:103D5E00F070CB90056BE004F080C31258C4900550
:0B3D6E0069E004F0A3E004F0023C2038
:013D79002227
:10480600A2AFE433900541F0A3E58EF0A3E589F06D
:10481600A3E58DF0A3E58BF0A28EE433A3F090041C
:10482600D4E0FF900547E4F0A3EFF0E07F00FE90B0
:104836000547F0A3EFF09004D3E0FDEDFF900547A8
:10484600EEF0A3EFF0C2AF9004D2740FF0125AE468
:104856009004D2E075F021A42400F974A835F0FA8A
:1048660090054974FFF0A3EAF0A3E9F0E4A3F09001
:104876000547E0FCA3E0FFECFD9004D5E0FBE4F582
:104886002CD20C12423090054DEFF0FD900549A355
:10489600E475F001123825FEAFF0124E3790054848
:1048A600E004F07006900547E004F090054CE00443
:1048B600F0E0C3942140B81258C49004D2E004F04A
:1048C600E0C3941E4087125497900541E024FF925E
:0148D600AF32
:0148D70022BE
:10472B00A2AFE433900541F0A3E58EF0A3E589F049
:10473B00A3E58DF0A3E58BF0A28EE433A3F09004F8
:10474B00D4E0FF900549E4F0A3EFF0E07F00FE908A
:10475B000549F0A3EFF09004D3E0FDEDFF90054980
:10476B00EEF0A3EFF0C2AF9004D2740FF09004D22E
:10477B00E0FFC3941E507875F021EFA42400F5825E
:10478B00E5F034A8AF8290054BF0A3EFF0E4900571
:10479B0047F0A3F0900549E0FCA3E0FFECFD90048B
:1047AB00D5E0FB90054BE475F00112382585F082BE
:1047BB00F583E493F52CC20C12423090054AE004C9
:1047CB00F07006900549E004F0900548E004F070A5
:1047DB0006900547E004F0C3900548E0942190054E
:1047EB0047E0940040AE9004D2E004F00247781208
:0A47FB005497900541E024FF92AFAF
:014805002290
:10423000C20D20C3FD20C5FAC2C4D2C5E490054F0B
:10424000F090054EF030C3FD30C3FDE4900551F011
:10425000E5C154F8F0E0FE64086004EEB4101A9072
:10426000054FE0B40105EB44018003EB54FEF5C2B9
:1042700090054E7401F002432C900551E0FEB418F5
:104280000F8DC290054E7402F0C2C4C2C502432C09
:10429000EEB420028051EE6428704490054EE0FE9A
:1042A000B4020B8FC27403F0C2C5C2C4807EEEB4E8
:1042B000031E300C09D2C590054F7401800D852C6A
:1042C000C2C2C590054E7404F0E4A3F0C2C4805C81
:1042D000EE64047057D2C490054E7405F0804D9082
:1042E0000551E0FEB4300FD2C4D2C590054E74081B
:1042F000F0E4A3F08036EEB43802802CEEB4400631
:10430000C2C2C2C58026EEB44802801CEEB4500280
:104310008004EEB45812D2C490054E7407F0900594
:1043200050E5C2F0C2C28004D2C4D2C5C2C3900557
:104330004EE0FE64076008EE6405600302424890A8
:044340000550E0FF45
:014344002256
:083FA4004105110041052A004E
:10597500AF84E4F584C2C343E60243F60275C3016E
:0B59850075C04475CF8E43C3018F84B2
:0159900022F4
:105497007E057F1690050BEEF0A3EFF0900512EE58
:1054A700F0A3EFF0900509EEF0A3EFF07E057F2B58
:1054B70090050FEEF0A3EFF0900514EEF0A3EFF0D8
:0D54C70090050DEEF0A3EFF0C21F02597525
:10554900900512E475F00112382585F082F583EF94
:10555900F0900512E475F00112382585F082F58383
:10556900EDF0900512E0B4050FA3E0B42A0A900506
:09557900127405F0A37416F0226F
:075ADD00C21FC2C4D2C522A2
:104BD700201F55D21F900514E475F0011238258562
:104BE700F082F58374FFF07C057D3F900514E0B5F6
:104BF700040FA3E0B5050A9005147405F0A3742B00
:104C0700F0900514E475F00112382585F082F583DC
:104C1700E4F0900514E0B5040FA3E0B5050A90058C
:104C2700147405F0A3742BF0900514E475F00112C9
:104C3700382585F082F583E4F07C057D3F900514E7
:104C4700E0B5040FA3E0B5050A9005147405F0A3B9
:104C5700742BF0900514E475F00112382585F08265
:104C6700F583EFF0900514E0B5040FA3E0B5050A4E
:0D4C77009005147405F0A3742BF07F01224A
:1057230090050BE0FCA3E0FD900509E0B50408A398
:10573300E0B505037F002290050BE0FCA3E0F582B2
:0C5743008C83E0B507037F01227F002269
:1056600090050CE004F0700690050BE004F0900546
:105670000BE475F00112382585F082F583E0FF9088
:10568000050BE0B4050FA3E0B42A0A90050B7405DE
:05569000F0A37416F008
:0156950022F2
:065AF0007FFF1257232284
:065AF600E4FF1257232219
:045AFC00E4F07FF75C
:015B00002282
:031A1800022B3C62
:102B3C00C0E0C0F0C083C082C0D075D000C000C05F
:102B4C0004C005C006C007E5C154F812390D2DAA02
:102B5C00002B97082B97102BE5182C31202C3E2896
:102B6C002CC7302CDB382CF1502CF1582D0C602C50
:102B7C00FB682D0C702CFB782D1C802D59882D1C7E
:102B8C00902D59982D75A000002DE9C2C590050E09
:102B9C00E004F0700690050DE004F07E057F3F9098
:102BAC00050DE0B5060FA3E0B5070A90050D7405F9
:102BBC00F0A3742BF090050DE475F0011238258507
:102BCC00F082F583E0F5C290050DE06E7003A3E092
:102BDC006F6003022DE9022CBA90050EE004F07030
:102BEC000690050DE004F07E057F3F90050DE0B5E5
:102BFC00060FA3E0B5070A90050D7405F0A3742B1E
:102C0C00F090050DE475F00112382585F082F583FE
:102C1C00E0F5C290050DE06E7003A3E06F60030257
:102C2C002DE9022CBA90050FE0FFA3E090050DCF23
:102C3C008019900514E0FEA3E0FF90050DE0FCA3C5
:102C4C00E0FDB50711ECB5060DA3EEF0A3EFF0C255
:102C5C00C5D2C4022DE98D828C83E0B4FF07C2C4B7
:102C6C00D2C5022DE990050EE004F0700690050D1A
:102C7C00E004F07E057F3F90050DE0B5060FA3E064
:102C8C00B5070A90050D7405F0A3742BF090050D93
:102C9C00E475F00112382585F082F583E0F5C290D9
:102CAC00050DE06E7003A3E06F6003022DE9900543
:102CBC000D7405F0A3742BF0022DE990050FE0FFC5
:102CCC00A3E090050DCFF0A3EFF0D2C4022DE99054
:102CDC00050FE0FFA3E090050DCFF0A3EFF0D2C4F9
:102CEC00D2C5022DE9ADC2E4FF125549022DE9907F
:102CFC00050FE0FFA3E090050DCFF0A3EFF0D2207D
:102D0C00ADC27FFF1255499005117401F0022DE9F7
:102D1C00900511E06006E5C264F0600690052AE0BB
:102D2C00601C90052A7401F0900509E0FFA3E09067
:102D3C000512CFF0A3EFF0AFC2125B008007ADC25B
:102D4C00E4FF125549900511E4F0022DE9900509B4
:102D5C00E0FFA3E0900512CFF0A3EFF090052AE07E
:102D6C006003125AFCD2C48074900512E0FFA3E0F9
:102D7C00900509CFF0A3EFF090052AE06003125AFA
:102D8C00FC302059900514E0FEA3E0FF90050DE007
:102D9C006E7003A3E06F6045D2C5C220803F9005E2
:102DAC000FE0FFA3E090050DCFF0A3EFF090050925
:102DBC00E0FFA3E0900512CFF0A3EFF090052AE01E
:102DCC006003125AFCD2C4900514E0FEA3E0FF90FD
:102DDC00050DE06E7003A3E06F6002D2C5C2C3D0D4
:102DEC0007D006D005D004D000D0D0D082D083D06C
:042DFC00F0D0E03201
:1056C90090050FE0FEA3E0FF90050DE0FCA3E0FDCF
:1056D900B50719ECB50615900514E0FEA3E0FFED3A
:0E56E900B50709ECB5060520C502D322C32281
:0E5A7E0000010002000400080010002000409B
:103FAC000265003241058C0041058D0041057B0006
:103FBC0041058F0041058E0041058B0041057600BF
:103FCC0041057500410584004105850041058600C9
:103FDC0044057C0000000044057700000000440507
:103FEC00870000000044058000000000015F000114
:023FFC00600162
:1039330090044EA3E0FF30E00F9004D0E0FBA3E03F
:10394300900434CBF0A3EBF0900435E02400F55958
:10395300900434E03480F558EF30E50F9004A4E090
:10396300FFA3E090043ECFF0A3EFF090043EE0FE0F
:10397300A3E07802CEC313CE13D8F9F5578E569031
:103983000575E0C39405500E90058CE06020E56654
:103993006432456560189004FDE0FEA3E0FFC3E4D4
:1039A3009FF555E49EF554E4F556F55780189004B9
:1039B300C4E06480FEA3E0FF9004FEE02FF5559081
:1039C30004FDE03EF55490058CE0600AE566643240
:1039D3004565600280499004C8E0C4F854F0C868A3
:1039E300FCA3E0C4540F48FD9004C8E0C313FEA336
:1039F300E0132DFDEE3CFC9004C8E01313543F7E0E
:103A0300002DFDEE3CFC30E7047C7F7DFF9004F944
:103A1300E0FEA3E0FFC3ED9FFDEC9EFC30E703E473
:103A2300FCFD75C30E8554C28555C1E556C313FE0F
:103A3300E557138E92F5918558C28559C18C928DA5
:103A43009175C27F75C1FF856D92856E91C281C2EA
:103A530081C281ACCFADCE90057BE030E03075C341
:103A63000E75C27F75C1FF8C928D918577C2857863
:103A7300C1E563C4F854F0C868FEE564C4540F4854
:103A83008E92F591C281C281C281ACCFADCEC3EC1F
:0D3A9300648094805003E4FCFD8C718D7202
:013AA0002203
:1018DC00AB72AA7175C3038AC28BC17592007591E4
:1018EC0008C281C281859654859555E55564074596
:1018FC00547068F557755640EA540FFCEB54F0756C
:10190C00C3038CC2F5C1759208759100C281C28166
:10191C00AC96AD95743C2DF582742A3CF583E4931A
:10192C007A0075C3018AC2F5C1759200759140C2E7
:10193C0081C281AA94AB93EB4257EA42567A377B29
:10194C000075C3018556C28557C18A928B91C2819D
:10195C00C281AA96AB958A6B8B6C22E4F557E55540
:10196C0025E0FFE55433FE747E2FF582745A3EF564
:10197C0083740193F556EA540FFCEB54F075C303D2
:10198C008CC2F5C1759208759100C281C281AC966A
:10199C00AD95743C2DF582742A3CF583E4937A0062
:1019AC0075C3018AC2F5C1E55525E0FFE55433FE48
:1019BC00747E2FF582745A3EF583E493FE74019382
:1019CC008E92F591C281C281AA94AB93EB4257EAF5
:1019DC0042567A377B0075C3018556C28557C18A3A
:1019EC00928B91C281C281AA96AB95EAA2E713FAB7
:0619FC00EB138A6BF56C91
:011A020022C1
:104C840090044EE0FCA3E0FDEC30E30F9004BCE0A4
:104C9400FFA3E090044ACFF0A3EFF090044AE0F5BC
:104CA40054A3E0F5559004B4E0FEA3E07802CEC32B
:104CB40013CE13D8F9FF900503E0FAA3E0FBC3EF8A
:104CC4009BF557EE9AF556EC30E20F9004BEE0FFE8
:104CD400A3E0900448CFF0A3EFF0900448E0F55827
:104CE400A3E0F55975C30EE42555FFE5543480F56A
:104CF400C28FC185569285579175C27F75C1FFE5F4
:104D040058C313FEE559138E92F591C281C281C234
:104D140081AFCEAECFC3EE648094805003E4FEFF37
:044D24008E638F64A7
:014D28002268
:10343900900576E0C3940550189004C2E06480FEBC
:10344900A3E0FF900500E02FFF9004FFE03EFE801F
:103459000F9004FFE0FEA3E0FFC3E49FFFE49EFE9C
:103469008E548F5590044EE0FCA3E0FD30E40F909C
:1034790004A2E0FFA3E090043CCFF0A3EFF0900496
:103489003CE0FEA3E07802CEC313CE13D8F9F5577A
:103499008E56ED30E20F9004CEE0FFA3E0900438A1
:1034A900CFF0A3EFF0900439E02400F559900438E7
:1034B900E03480F5589004C6E0FCA3E0FDECC4F8C4
:1034C90054F0C868FAEDC4540F48FBECC313FEED81
:1034D900132BFDEE3AFC9004C6E01313543F7E0013
:1034E9002DFFEE3CFE900573F0A3EFF0EE30E70AF6
:1034F900900573747FF0A374FFF09004FBE0FEA3C2
:10350900E0FFC3900574E09FFF900573E09EFEF015
:10351900A3EFF0EE30E707E4900573F0A3F0900510
:093529008EE0640260030235AF7C
:1035320085715A85725BC3E56A94FFE569943F40E1
:1035420027E56A2401FFE56934C0FEEF255BF55BE0
:10355200EE355AF55AD3E55B94FFE55A947F401E47
:10356200755A7F755BFF8016C374FF956AFF743FBF
:103572009569FEC3E55B9FF55BE55A9EF55A75C3F7
:103582000E8554C28555C18556928557918558C27C
:103592008559C1900573E0FEA3E0FF8E928F91756D
:0B35A200C27F75C1FF855A92855B91C6
:1035AD00802D75C30E8554C28555C185569285579C
:1035BD00918558C28559C1900573E0FEA3E0FF8E39
:1035CD00928F9175C27F75C1FF856992856A91C28F
:1035DD0081C281C281900573E5CFF0A3E5CEF09055
:1035ED000573E030E707E4900573F0A3F0900573E1
:0735FD00E0F56FA3E0F5709B
:0136040022A3
:103AA100AB70AA6F75C3038AC28BC1759200759101
:103AB10008C281C281859654859555E555640745AF
:103AC100547066F557755640EA540FFCEB54F07587
:103AD100C3038CC2F5C1759208759100C281C28180
:103AE100AC96AD95743C2DF582742A3CF583E49334
:103AF1007A0075C3018AC2F5C1759200759140C201
:103B010081C281AA94AB93EB4257EA42567A377B42
:103B11000075C3018556C28557C18A928B91C281B6
:103B2100C281AA96AB95023BC2E4F557E55525E063
:103B3100FFE55433FE747E2FF582745A3EF583748B
:103B41000193F556EA540FFCEB54F075C3038CC294
:103B5100F5C1759208759100C281C281AC96AD958F
:103B6100743C2DF582742A3CF583E4937A0075C385
:103B7100018AC2F5C1E55525E0FFE55433FE747EA7
:103B81002FF582745A3EF583E493FE7401938E926D
:103B9100F591C281C281AA94AB93EB4257EA425696
:103BA1007A377B0075C3018556C28557C18A928BCE
:103BB10091C281C281AA96AB95EAA2E713FAEB13EF
:103BC100FB90058EE014603E14603D2402703DAA16
:033BD1006FAB7067
:103BD40075C3038AC28BC18A928B91C281C28185CB
:103BE400965885955975C3038558C28559C17592F0
:103BF40001759100C281C281AA96AB950BBB0001ED
:013C04000AB5
:083C0500800280008A678B68D1
:013C0D002294
:10464B0090044FE030E70F9004A6E0FFA3E0900446
:10465B0042CFF0A3EFF0900442E0F554A3E0F55500
:10466B00E42555F55574803554F5549004B8E0FEA7
:10467B00A3E07802CEC313CE13D8F9FF900505E063
:10468B00FAA3E0FBC3EF9BF557EE9AF55690057B2B
:10469B00E030E12F75C30E8554C28555C185569206
:1046AB0085579175C27F75C1FFE575C313FEE5761E
:1046BB00138E92F5918577C28578C1856392856457
:1046CB0091802175C30E8554C28555C1855692853F
:1046DB00579175C27F75C1FFE575C313FEE5761360
:1046EB008E92F591C281C281C281ACCFADCEC3ECAB
:1046FB00648094805003E4FCFD7466F554F55575A5
:10470B00C3038CC28DC1855492855591C281C281E0
:0F471B00AC96AD9574992DFD74193CF5618D62C6
:01472A00226C
:04520600AD07AC063E
:10520A009004B0E0FEA3E07806CEC313CE13D8F91B
:10521A002401FFEE34FE900573F0A3EFF030052D64
:10522A00900573E0FEA3E0FFD39400EE64809480BF
:10523A00400FEF2DFDEE3CFC30E7127C7F7DFF80B6
:10524A000CEF2DFDEE3CFC30E703E4FCFDAE04AFB1
:01525A00054E
:01525B002230
:104A6D0090044FE030E60F9004ACE0FFA3E090041B
:104A7D0040CFF0A3EFF0900440E0F554A3E0F555DE
:104A8D009004B6E0C313FEA3E013FF900501E0FA16
:104A9D00A3E0FBC3EF9BF557EE9AF55690057BE02F
:104AAD0030E23575C30EE42555FFE5543480F5C26B
:104ABD008FC185569285579175C27F75C1FFE5737C
:104ACD00C313FEE574138E92F5918577C28578C177
:104ADD00856392856491802775C30EE42555FFE5A6
:104AED00543480F5C28FC185569285579175C27F1A
:104AFD0075C1FFE573C313FEE574138E92F591C274
:104B0D0081C281C281ACCFADCEC3EC6480948050A4
:084B1D0003E4FCFD8C798D7AA4
:014B2500226D
:10326A00C210E55F1470030233311470030233593C
:10327A0014700302337E1470030233A524EB700327
:10328A000233B51470030233E024E87003023402F7
:10329A002432600302340F90044FE030E10F9004AF
:1032AA00CCE0FFA3E0900436CFF0A3EFF090058CBA
:1032BA00E0604EE56664324565602E9004DAE0C34C
:1032CA0013FEA3E013251AFDE5193EFCE56624CE9C
:1032DA00FFE56534FFFEEF7802C333CE33CED8F96B
:1032EA002DF56EEC3EF56D802F900436E0C313FE8B
:1032FA00A3E013251AF56EE5193EF56DAF6EFE8053
:10330A0010900436E0C313F56DA3E013F56EFFAE1B
:10331A006D1252068E6D8F6EE56D30E705E4F56D20
:10332A00F56E055F02341190044FE030E30F90040C
:10333A00CAE0FFA3E090043ACFF0A3EFF090043A7A
:10334A00E0C313F569A3E013F56A055F023411902F
:10335A00044EE030E00F9004AEE0FFA3E090044496
:10336A00CFF0A3EFF0900444E0F573A3E0F5740501
:10337A005F02341190044EE030E10F9004A8E0FFA0
:10338A00A3E0900446CFF0A3EFF0900446E0C31305
:10339A00F575A3E013F576055F806CAF84E4F584D8
:1033AA00D2EC85109B8F84055F805C9005A2E0704B
:1033BA00231256F7EF601D90059CE0FF30E70F20BF
:1033CA001C0C64F060089005A27402F08006900557
:1033DA00A27401F0055F9005A2E0B4021990058C71
:1033EA00E0600E7B017A05799B124561EF24FF921A
:1033FA0010E49005A2F0055F0560E5607002D22234
:10340A00E4F55F8002055FE55F30E10930E006120E
:10341A00464B023933E55F30E1061234390218DCD3
:0E342A00E55F30E003023AA1124C84124A6DB5
:013438002271
:03000000020C00EF
:03000300021A03DB
:03000B00021A06D0
:03001300021A09C5
:03001B00021A0CBA
:03002300021A0FAF
:03002B00021A12A4
:03003300021A1599
:03003B00021A188E
:03004300021A1B83
:03004B00021A1E78
:03005300021A216D
:03005B00021A2462
:03006300021A2757
:03006B00021A2A4C
:03007300021A2D41
:03007B00021A3036
:03008300021A332B
:03008B00021A3620
:03009300021A3915
:03009B00021A3C0A
:0300A300021A3FFF
:100C0000787FE4F6D8FD9000007F007E20E4F0A31A
:0A0C1000DFFCDEFA75817E020C5550
:100C1A00020C9AE493A3F8E493A34003F68001F24A
:100C2A0008DFF48029E493A3F85407240CC8C333DB
:100C3A00C4540F4420C8834004F456800146F6DFAA
:100C4A00E4800B0102040810204080903EDBE47E21
:100C5A00019360BCA3FF543F30E509541FFEE4939F
:100C6A00A360010ECF54C025E060A840B8E493A366
:100C7A00FAE493A3F8E493A3C8C582C8CAC583CA91
:100C8A00F0A3C8C582C8CAC583CADFE9DEE780BE49
:013FFE0000C2
:1037B700BB010689828A83E0225002E722BBFE0210
:0937C700E32289828A83E4932243
:1037D000BB010CE58229F582E5833AF583E02250AE
:1037E00006E92582F8E622BBFE06E92582F8E222F8
:0D37F000E58229F582E5833AF583E4932212
:1037FD00BB010689828A83F0225002F722BBFE01AB
:02380D00F322A4
:10380F00C5F0F8A3E028F0C5F0F8E5821582700244
:06381F001583E038F022E1
:10382500A3F8E0C5F025F0F0E58215827002158356
:06383500E0C838F0E822B3
:10383B00BB0110E58229F582E5833AF583E0F5F0CB
:10384B00A3E0225009E92582F886F008E622BBFEA8
:10385B000AE92582F8E2F5F008E222E5832AF583EE
:08386B00E993F5F0A3E99322B3
:10387300BB010A89828A83F0E5F0A3F0225006F7A0
:0F38830009A7F01922BBFE06F3E5F009F319229D
:10389200F8BB0111E58229F582E5833AF583E8F068
:1038A200E5F0A3F0225009E92582C8F608A6F02225
:0D38B200BBFE09E92582C8F2E5F008F2220C
:1038BF00EB9FF5F0EA9E42F0E99D42F0EC6480C880
:0638CF0064809845F02220
:1038D5007401FF3395E0FEFDFC080808E6CF2FF6DE
:1038E50018E6CE3EF618E6CD3DF618E6CC3CF622B7
:0C38F500ECF0A3EDF0A3EEF0A3EFF02246
:0C390100A42582F582E5F03583F58322D1
:10390D00D083D082F8E4937012740193700DA3A349
:10391D0093F8740193F5828883E47374029368605D
:06392D00EFA3A3A380DF5D
:00000001FF
